:020000040800F2
:100000000002002081040008ED040008FD0400083F
:10001000C5060008D5060008E50600080000000037
:100020000000000000000000000000004104000883
:10003000F506000800000000250400080B02000877
:100040000B0200080B0200080B0200080B0200085C
:100050000B0200080B020008C5130008C5130008B6
:10006000C5130008C5130008C51300080B020008DB
:100070000B0200080B020008E51100080B02000843
:100080000B020008B91100080B0200080B0200085F
:100090000B0200080B0200080B020008C513000841
:1000A0000B0200080B0200080B0200080B020008FC
:1000B000B51600080B0200080B0200080B0200082E
:1000C0000B0200080B0200080B0200085534000860
:1000D000613400080B020008AD110008D9110008B6
:1000E000C51300080B0200080B0200080B020008F1
:1000F0000B0200080B0200080B0200080B020008AC
:100100000B0200080B020008BB1600080B020008D7
:100110000B0200080B0200080B0200080B0200088B
:100120000B0200080B0200080B0200080B0200087B
:100130000B0200080B0200080B0200080B0200086B
:100140000B0200080B0200080B0200080B0200085B
:100150000B0200080B0200080B0200080B0200084B
:100160000B0200080B0200080B0200080B0200083B
:100170000B0200080B0200080B0200080B0200082B
:100180000B0200080B02000800F0C4BA7047000020
:1001900070B50C46064600F061F9094B094A1D6826
:1001A0002C44944202D8084A944207D20C2333606C
:1001B0004FF0FF3500F05AF9284670BD1C60F9E792
:1001C00000020020000002200C28002019461046E2
:1001D00000F0ACBA1946104600F0B0BA1323036021
:1001E0004FF0FF307047132303604FF0FF3070472C
:1001F000132303604FF0FF30704702294FF00003D4
:1002000003608CBF00200120704700F07BBA000023
:10021000114B70B500241C60104B114D18682E68EE
:1002200000F09CF80F4B53F820301B68A3F1080234
:1002300096420FD026B13179092904BF0A213171C4
:10024000092103F8041C33F9021C074B2A601980AA
:10025000012070BD204670BDC0020020B402002005
:10026000BC020020C8020020B8020020082930B5D6
:1002700003791AD9082B14D842791A4B53F8225013
:1002800000F108047DB12D68856053F822502C6080
:1002900043F82240144A44790123A34014682343BD
:1002A0001360017130BD8460F2E7082BF9D94579FC
:1002B0000C4B53F825203AB11468A2420BBF002220
:1002C000246843F825201460427953F82230002B2B
:1002D000E7D1054C012303FA02F2236823EA020363
:1002E0002360DEE7C8020020B402002008B50A4BF4
:1002F0001B681A79082A02D95B7983420AD900F06F
:10030000B8F818B1054B01221A6008BDBDE80840D5
:1003100000F080B808BD00BFBC020020C002002071
:1003200008B500F09BF8094B094A1B88094D1BB220
:10033000002442F82340084A286813682146013BFC
:100340001360FFF793FF2C6000F060F8B802002004
:1003500008030020BC020020C40200200023C207C2
:1003600001D51846704740080133F8E7134423F0DD
:10037000030310B54FF077321C1F43F8042C6207BB
:1003800042BF4FF0883243F8082CA3F108044FF025
:10039000807304E909000F4B44F80C3C002344F837
:1003A000103C032344F8143C2246022344F8183C32
:1003B000012344F81C3C42F8201D0B2342F8043D65
:1003C000013B032BFAD120466FF0020340F8443D75
:1003D00010BD00BF210300080548064A064B01680E
:1003E000914201D1984201D3181A70470430F6E7C0
:1003F00000000020FEE7FEE700020020EFF3088087
:1004000070470000004870470000002000F02AF804
:1004100001DFFEE7024A536843F0805353607047A0
:1004200000ED00E0EFF3098020E9F00F40F804ED63
:1004300002490968086000F003F80000BC020020CF
:10044000FFF7E6FE04480068016801C9B1E8F00F53
:1004500081F3098800470000BC020020EFF3108000
:1004600072B6704762B6EFF31080704780F3108861
:100470007047EFF30580C0B27047704770470000C7
:1004800008B5FFF7FAFF6A46114B1249934213D39E
:10049000114A124B12498B4211D3124B124A0021BE
:1004A000934211D3FFF7EAFF00F022FB03F0D8FCE0
:1004B000BDE8084000F076BB43F8041BE6E752F8BD
:1004C000040F43F8040BE6E743F8041BE8E700BF1A
:1004D00000000020FEE7FEE76C5300080002002049
:1004E000B4020020B40200200C28002008B5024904
:1004F000042000F01BFB00BF8D4F00080D490E4A81
:100500000E4B6846904203D8984201D9002102E080
:1005100009468D46012104207246024202D1EFF3C2
:10052000088001E0EFF309802DE9F00F6B4600F041
:1005300007F800BF00020020000002206005002034
:100540002DE9F04F9A46494B8FB093469A6B039230
:100550005A6B04929F6ADA6A05921A6BDB6B0793F7
:10056000434B06921A68434B9A420446884602D08F
:10057000414803F02FFDB8F1000F4ED03F4803F083
:1005800029FD00252E463E4803F024FD39463D480E
:1005900003F0ACFC05993C4803F0A8FC06993B48E5
:1005A00003F0A4FC07993A4803F0A0FC3A0403D5F1
:1005B0000399384803F09AFC3B0603D50499364862
:1005C00003F094FC354803F005FD5946344803F028
:1005D0008DFCB8F1000F1BD1324803F0FBFC314613
:1005E000314803F083FC6946304BC91A03D54942B0
:1005F0002F4803F07BFC20468268C36801698C4663
:1006000041698E46AD46514691E8F00F4168006859
:1006100001BE2849052000F089FA94E80E00E06840
:10062000D4F81C9008902069099060690A9019F428
:10063000007F2148A6690D930CBF04F1200504F149
:1006400024050C920B9103F0C5FC089B00930BA9A9
:100650000EC91A4803F04AFCCDF8009033460A9AB6
:100660000999174803F042FC8DE700BF00ED00E058
:1006700000000020FEE7FEE7864D00089C4D0008C4
:10068000614E00086A4E00087A4E00088A4E000843
:100690009A4E0008AA4E0008BA4E0008CA4E00083A
:1006A000CF4E0008E14E0008124F0008580100200C
:1006B0003A4F0008674F0008CB4D0008E64D000890
:1006C000234E000808B50249062000F02FFA00BFAB
:1006D0007A4F000808B50249072000F027FA00BF4A
:1006E000544D000808B50249082000F01FFA00BF69
:1006F000994F000808B50249092000F017FA00BF19
:10070000664D000808B502490A2000F00FFA00BF44
:10071000784D0008034B044A4FF4E131002000F00B
:100720007FBC00BF04020020ED0E00080A4601460F
:10073000014800F0E6BB00BF0402002010B50A46E5
:100740000C460146002000F015FC204610BD00209C
:1007500000F052BF034B1968024611B9084600F079
:100760002BBF7047CC03002010B5094A136843B172
:100770009C6881688C4207D303D15C6841688C42D5
:1007800002D90360106010BD1A461B68EFE700BF76
:10079000D4030020F0B51F4E1F4D33681F4C0133AA
:1007A00033601F4B00201A6818602B6822601946BE
:1007B0000746B64621B1DEF800C08E68664503D90B
:1007C00000B1296027B9F0BD0F4601200968F1E7A3
:1007D00000213960DAB163B151685868814294BF31
:1007E00011461946084612681B6822B90360216049
:1007F000F0BD1146F6E70BB90260F8E755685E6890
:10080000B54294BF15461D4605602846EBE72360B8
:10081000F0BD00BFD0030020D4030020DC03002083
:10082000D80300202DE9F0412C4F2D4C01233B60D3
:10083000236893B9FFF7AEFFFFF789FF0130FBD0C4
:1008400000254FF0000823685BB9FFF780FF854261
:1008500024D9FFF79FFF0025F5E7FFF778FF05464E
:10086000EFE75E68FFF773FF854204D8864202D93E
:10087000361A132EE9D823685E68FFF768FF8542B1
:1008800001D88642F7D823681A682260C3F804802A
:10089000C3F80880DA6818699047D4E723686BB119
:1008A0005E68FFF754FF063E14308642CBD3002328
:1008B0003B603046BDE8F041FFF74CBFFFF747FF14
:1008C00085420646C5D810F1140F04D3FFF73FFF49
:1008D0008642FBD9BDE74FF0FF36E8E7CC030020A6
:1008E000DC030020144B1A6882420FD112681A6090
:1008F0001AB150680638FFF72DBF4FF0FF30FAE706
:10090000904202D102681A60704713461A68002AA2
:10091000F6D10A4A13681BB9094A13683BB97047F4
:10092000984202D10368136070471A46F2E7984272
:10093000F8D01A46F1E700BFDC030020D8030020FE
:10094000D403002008B500231846054A054900F0E5
:1009500079FE4FF0FF30BDE80840FFF7FBBE00BF57
:100960002508000840420F00F8B504460D46FFF781
:10097000EEFE002385420646236011D3A5F10A034B
:1009800083420DD20A35FFF7E2FE8542FBD3FFF723
:10099000DEFE8542FBD8E368206998470020F8BD59
:1009A000FFF75CFD63680746002B33D1A368002B7B
:1009B00030D11A4B65601A681B68B54238BF0132E6
:1009C000A260A2689A4206D92046FFF7CDFE3846BB
:1009D000FFF74CFDE2E7B5420FD9114B19461A68F3
:1009E00012B15068854213D222601C600B689C4291
:1009F000EDD1A81FFFF7AEFEE9E70A4A136813B16D
:100A000059688D4202D223601460E0E71A46F5E788
:100A10001346E4E72046FFF765FFCAE7D00300204E
:100A2000DC030020D803002038B50446FFF716FD8C
:100A30006368054633B9A36823B92846BDE8384042
:100A4000FFF714BD2046FFF74DFFF6E7C36870B50A
:100A500004460D46C3B1FFF7E7FF092D0CD8FFF799
:100A600076FE0646FFF773FE801B8542FAD8E368E0
:100A70002069BDE870401847FFF769FE2918204635
:100A8000BDE87040FFF770BF70BD00002DE9F04772
:100A900004460E4690461AB9BDE8F047FFF7D6BFA8
:100AA000FFF7DCFC63680746E3B9A368D3B9DFF856
:100AB0003CA0FFF74CFEDAF800508146FFF747FEF6
:100AC0008145F6D8304408EB0502864288BF0132E2
:100AD0006060A2602046FFF747FE3846BDE8F04759
:100AE000FFF7C4BC2046FFF7FDFEE0E7D00300207F
:100AF00008B50121094800F085FB0121084800F0F4
:100B000081FB0121074800F07DFB0121064800F030
:100B100079FBBDE8084000F033B900BF0D0C02407E
:100B20000C0C02400E0C02400F0C024008B50E4B9C
:100B30001A680C469AB9012203281A6003D171463B
:100B40000A4803F0D3F92146094803F0CFF900F031
:100B500061FC084803F0CAF9074803F0C7F9FFF73A
:100B60007DFC00F0FBF800BFE0030020BF4F000851
:100B7000C34F0008EB4F0008DF4F000808B50348DB
:100B800003F0B4F900F0F2FD002008BDED4F0008BD
:100B900008B5034C2368012000F072F9FAE700BFA2
:100BA000E40400201FB5FFF759FC0E4B0E481B68EC
:100BB000029300240D4B00930F220C234FF48071FD
:100BC000019400F055F80A4B0A481B6802930A4B3F
:100BD000009307220C234FF4C061019400F048F801
:100BE000FFF714FC18020020E4030020910B00081A
:100BF0001C020020E80400207D0B000808B5FFF768
:100C00002DFC094B1B681A79082A07D95A79074B1A
:100C100053F8221011B1096843F82210FFF726FC9F
:100C2000BDE80840FFF7F6BBBC020020C802002068
:100C300038B50B79082B03D908490320FFF776FF55
:100C40004C7901F10802036813B98B60026038BD6A
:100C500013F8035CAC42F8D31846F4E7AD4F000834
:100C6000031F53F8042F9A42FBD0181A7047000054
:100C70000F2A2DE9F74F05468B4691469A4633D801
:100C800010F003031BBFC3F10403ED180B46CB1A8E
:100C9000303B23F003031AF0080F05EB030419D0CF
:100CA0002A46A24213D30193FFF7D8FB2949019B9F
:100CB0008046012251F8226017B2C6B10132212AC2
:100CC000F8D14046FFF7D2FB6FF08A073DE0126093
:100CD0000432E6E72D60E6E701212046FFF7C6FA79
:100CE0004046FFF7C3FB30E06FF015072DE041F8F9
:100CF00022400C98E7802A460D99FFF737FB0E9BA0
:100D0000154AA3624FF0FF33E3611368206001339B
:100D10001AF0010F6562C4F82CB084F805902671B2
:100D2000A660E66026616661A66126621360D3D183
:100D30000A212046FFF79AFA1AF0040FD0D1404654
:100D4000FFF794FB4846FFF7D1FA384603B0BDE8F9
:100D5000F08F00BF08030020C402002008B5EFF3A5
:100D60000581C1F3080119B11039044803F0BEF838
:100D700000BE042000F084F8FBE700BF3A500008F2
:100D800010B53C4C01F0D2FB0022A260236823F096
:100D9000867323F480332360E260236843F4803356
:100DA000236023689803FCD54FF08051002000F0A9
:100DB000B1FB314A136843F400431360A36823F086
:100DC000F003A360A368A360A36823F46043A36057
:100DD000A36843F40043A360A36823F4E053A36033
:100DE000A36843F4A053A36000236360636843F4E3
:100DF00080036360636843F008036360636843F4DF
:100E0000A843636063686360636843F0E0636360A2
:100E1000236843F08073236002F5E432136899017C
:100E2000FCD5164B00211960196841F40071196056
:100E3000196841F480611960196821F00F01196087
:100E4000196841F005011960936823F0030393606A
:100E5000936843F002039360064B19469A681207A1
:100E6000FCD51A6822F001021A600B689B07FCD4BB
:100E700010BD00BF0038024000700040003C02403E
:100E8000174B93F90010042806D8DFE800F0030799
:100E9000101C1C0000221A700846704701221A70AC
:100EA000104A136923F00403136130BFF4E70222F0
:100EB0001A700D4A136823F003031360094A13697B
:100EC00043F00403F0E703221A70074B1A6842F05C
:100ED0000E021A605A6842F480725A60EEE700BF50
:100EE0002002002000ED00E00070004038B504460C
:100EF000043000F0FAFB0546204601F0F1FA2846DE
:100F000038BDF8B504460E461746051D3A4631462B
:100F1000284600F0D5FB00B1F8BD0121204601F0C4
:100F2000AFFAF3E74209012300F01F0003FA00F0D3
:100F3000014B43F82200704700E100E0024B1B68C0
:100F40000BB1FFF75BBE7047C002002008B50B680D
:100F50009B0608D5064B496803EBC002C9B253F89B
:100F6000303050689847BDE80840FFF7E7BF00BF42
:100F7000F80A00202DE9F84306460C461546FFF70F
:100F800078FADFF8849078B118235E43254459F845
:100F90000630AC4201D1BDE8F8831A681206FCD5D0
:100FA00014F8012B5A60F4E7134F4FEA86084744C0
:100FB0000121384601F064FA182303FB06960F4816
:100FC000F17C0F4A0729D8BF024601F00701102023
:100FD00013FB0103D118ADB2CC604D60D158094864
:100FE00041F00101D1504044012101F049FA384655
:100FF000BDE8F84301F074BAF00A00200060024036
:1010000000640240E80A00204C500008034A1823FC
:1010100003FB00204168407C00F07CBA4C50000883
:1010200001282DE9F84F05460C4600F2A78018214B
:101030004143544F07EB01087E58534941F8302093
:1010400001EBC0014FF000094B60504B43F820907A
:101050004F48012140F8259000EB850001F010FA7F
:10106000D8F808B04946584600F0CCF8D8F80C90AB
:101070000121484600F0C6F898F810A0584651469D
:1010800000F066F95146484600F062F92846FFF73D
:10109000BDFF98F811302401002B4FD13D48B0FB23
:1010A000F4F002F015FD804602F0BAFE84B220464C
:1010B00002F012FD0146404602F058FC4FF0834119
:1010C00002F05EFD02F0ACFE240100F00F00A4B2BD
:1010D00004438023B46073610023336142F20C0344
:1010E000F360182303FB0573DC7C072C28DC4FF42A
:1010F0000011022000F00EFA274A1820102104F0F7
:10110000070310FB031300FB05702449057D90F9CC
:10111000120002EB030E41EA4561D150331DCEF8B7
:1011200008300023CEF81430FFF7FCFE062C0EDC4E
:1011300004F10B0040B2FFF7F5FE0EE01848AEE7F1
:101140004FF48001022000F0E5F9164AD5E7072C9C
:101150000AD1154B4FF400425A60F36843F0200364
:10116000F3600020BDE8F88F0C2C02DC04F13000A5
:10117000E0E70F2CF1DC04F13700DBE74FF0FF3044
:10118000BDE8F88F4C500008F80A0020F00A002053
:10119000E80A002080DE8002006002405004010066
:1011A00000BD01050064024000E100E001490020AB
:1011B000FFF7CCBE0044004008B5054B05484FF48E
:1011C0000012DA6001F08CF9BDE80840FFF7B6BE06
:1011D00000600240E80A002001490120FFF7B6BE86
:1011E0000048004008B5054B05484FF000629A6082
:1011F00001F076F9BDE80840FFF7A0BE00600240AC
:10120000EC0A0020F8B50D460126C0F3832120F03A
:101210000F0400F00F0706FA01F1022000F07AF93E
:1012200007FA06FE0323226803FA0EF3D8430240AE
:101230002260226805F0030101FA0EF111432160DA
:10124000E2681040E060E168C5F3810202FA0EF244
:101250000A43E2606268BE4022EA06026260626897
:10126000C5F30015BD4015436560A268B6B21343CF
:10127000A36000206683F8BD2DE9F04100F00F0463
:101280001746304A42F8343002EBC402069B5360E2
:1012900005468846C0F383264FF48041012000F0C4
:1012A00039F941462846FFF7ADFF042C264B28DCD0
:1012B000A11D01228A401A60012F244B2AD032D36B
:1012C000022F3AD004F00C0303F1804303F59C3362
:1012D00005F003059A68AD000F21A94022EA01023A
:1012E0009A609A6806FA05F515439D60012303FA92
:1012F00004F4164B5C611A6814431C600020BDE8BE
:10130000F081092C02DC4FF40002D4E74FF4807224
:101310005A60D1E79A68A7403A439A60DA6822EAAD
:101320000707DF60CEE799680122A24021EA0201A7
:101330009960D9680A43DA60C4E799680122A2403B
:101340001143F5E7080B002000E100E0003C0140FC
:1013500020F00F03F0B500F00F041D6867000326AE
:10136000BE4025EA06051D601D680222072C02FA10
:1013700007F242EA050294BF002401241A6003EB3D
:10138000840300F007001A6A80000F24844022EAD8
:1013900004021A621A6A01FA00F010431862F0BDE2
:1013A00020F00F0200F00F030120984080B210835C
:1013B000704720F00F0200F00F030120984080B228
:1013C000508370472DE9F0410F4D104F6E692A6828
:1013D000002416404FF0010808FA04F31E4206D01C
:1013E0006B6107EBC40357F8342058689047013409
:1013F000102CF1D1064B1B681BB1BDE8F041FFF783
:10140000FDBBBDE8F08100BF003C0140080B00209F
:10141000C00200202DE9F04F2D4B2E4A1B882E498B
:101420002E48DFF8CC90DFF8CCA0DFF8CCB08BB042
:101430000126ADF8243002F059FDFEF7CDFF054638
:10144000FEF7E0FF0446FEF7D9FF2A460090234648
:101450004FF40071224802F049FD25EAE5754FF48A
:10146000007759F826401CB394F80480E26A5AF8D1
:101470002830606A079317440692FFF7F1FB069A3B
:10148000B4F90610079B101A22680592626A04924A
:101490000390E26A02926279019209AAB8F1080FF8
:1014A000C8BF013200920544A26A584602F01EFDF0
:1014B0000136212ED5D10B4B02958DE888000A4AC2
:1014C0000A48194602F012FD0BB0BDE8F08F00BFCC
:1014D0007C5000087E5000088450000889500008A5
:1014E000CF50000855510008575100085B510008C3
:1014F000080300202402002019510008034B044A6D
:1015000000280CBF10461846704700BF00BD0105FB
:1015100080DE8002042808D8DFE800F0030A0F14F8
:1015200019000D4A136C19431164BFF34F8F7047B4
:10153000094B5A6C11435964F7E7074B1A6B114377
:101540001963F2E7044B5A6B11435963EDE7024B01
:101550009A6B11439963E8E7003802402DE9F8439C
:10156000124ADFF8508003010746D5582E69EB6810
:1015700000241E4008EBC0090223A3401E4209D0EC
:10158000EA68D9F8040022EA0303EB60214658F820
:10159000373098470134042CEED1054B1B681BB142
:1015A000BDE8F843FFF72ABBBDE8F883CC5100083B
:1015B000C0020020880B0020032910B516D80D4B5F
:1015C00000011C18185863681A4001F10C0300EB65
:1015D00083035A600269022303FA01F122EA01023D
:1015E0000261C3681943C160002010BD4FF0FF3095
:1015F00010BD00BFCC5100080001024B1B58586AB7
:10160000704700BFCC510008034B00011A58136803
:1016100043F0010313607047CC510008074B03EB04
:1016200000100121437B5AB203F01F0301FA03F3B8
:101630005209034941F82230704700BFCC510008DD
:1016400000E100E001282DE9F84305460F4629D8BE
:10165000164E1749040106EB040841F8302098F8AB
:101660000C9001EBC00148464B60D8F80810FFF71A
:1016700051FF3659D8F8043000243460484674606D
:10168000F362FFF73BFF0123B0FBF7F00138B062D4
:1016900073612846FFF7C2FF2846FFF7B5FF2046D3
:1016A000BDE8F8834FF0FF30BDE8F883CC51000867
:1016B000880B00200020FFF751BF0120FFF74EBF2D
:1016C00070B514461CB18568C3689D4201D1101BDA
:1016D00070BD86680568731C83604368013B3340B6
:1016E000013CEB5C01F8013BECE7C268436830B5B4
:1016F0008468121B9A4208D0C2680468013B1340F8
:10170000551CC560E154002030BD4FF0FF3030BDA6
:1017100037B500210E480F4C02F0E8FB0E490F4888
:1017200000F030F80D49204601F012F8002105467E
:101730000B4802F0DBFB002D07DB0094094B0A4845
:1017400002224FF4806101F08DF803B030BD00BF7C
:1017500000520008D00F0020EC510008980F002024
:101760004550000828520008980B002008B504488E
:1017700002F030FCFFF7E6F8FFF7CAFF002008BDD3
:101780003252000838B50C4B0446142240F8203B76
:101790000D4602F098FB082384F8363000210F2311
:1017A00084F8343084F837106A7894F82000BDE863
:1017B000384001F0A9BD00BF5C52000870B5044676
:1017C00086B000F081F9204600F04BFE03AE002108
:1017D000A176A1830C22304602F080FB304601F056
:1017E0007BFE082505F0070306AA1344715D13F874
:1017F0000C2C01354A400C2D03F80C2CF2D19DF82D
:101800000C3023F00103314643F00203082201A803
:101810008DF80C3002F057FB029A019B12BA1BBAEA
:10182000204600F0A5FCBDF8041049BA204689B254
:1018300000F08FFC2046232100F0CBFC20461A212B
:1018400000F0BAFC2046002100F0E0FC2046012216
:10185000202100F054FD204601224FF4807100F059
:101860004EFD204600224FF4005100F048FD204676
:1018700001224FF4804100F042FD002323738022B7
:101880002946204600F07DF80421204600F095F816
:10189000042100F0FD02204600F073F803212046E9
:1018A00000F08BF8032100F0F002204600F069F808
:1018B000082220460E2100F064F80F21204600F097
:1018C0007CF81621204600F094FD06B070BD10B5DE
:1018D000044600F0E2F80821204600F06EF80821E6
:1018E00000F08002204600F04CF80121204600F074
:1018F00064F80306F9D5C0F3801010BD10B590F858
:1019000037300133044680F83730204600F0B9F80C
:10191000A0F11103DBB2012BF7D9192818BF84F805
:1019200036001921204600F064FD022384F835308A
:1019300010BD70B51D4690F835306E1C134414462A
:1019400080F8353013460A46F1B200F054F86019B9
:1019500070BD10B5012300F135020021044600F0EE
:101960004AF802221146204600F00BF863683BB1AA
:10197000A28B120504D520460321BDE8104018476C
:1019800010BD70B5044690F820000D46164601F0D3
:1019900027FD606AFFF70DFD324645F0C0010023C8
:1019A00094F8200001F083FD606AFFF7F9FC94F8D9
:1019B0002000BDE8704001F023BD37B5044690F823
:1019C00020000D4601F00CFD606AFFF7F2FC0DF1FE
:1019D0000703002245F0800194F8200001F067FD24
:1019E000606AFFF7DDFC94F8200001F009FD9DF826
:1019F000070003B030BDF8B5044690F820000F464C
:101A000015461E4601F0ECFC606AFFF7D2FC3A4630
:101A10000023402194F8200001F049FD3346294677
:101A2000002294F8200001F021FD606AFFF7B8FC65
:101A300094F82000BDE8F84001F0E2BC10B504467F
:101A400090F8200001F0CCFC606AFFF7B2FC94F83B
:101A5000200000222021BDE8104001F0E1BC134627
:101A600090F820000A46002101F000BD10B50446A0
:101A7000406AFFF795FC94F82000BDE8104001F0A3
:101A8000BFBC08B590F834300F2B04D00121FFF70C
:101A900094FF00F01F03184608BD10B50446FFF779
:101AA000F0FF0F280FD1E06AFFF783FC00214FF40D
:101AB000967001F027FD01212046FFF77EFF00F020
:101AC0001F0084F8340010BD10B50446FFF7E5FF91
:101AD000206BFFF76EFC0021012001F013FD206B4D
:101AE000FFF75EFC00211A20BDE8104001F00ABD9E
:101AF00010B5032202210446FFF743FF2046FFF7FB
:101B0000C0FF0828FAD110BD38B50446FFF7C5FF5D
:101B10002046FFF7B6FFA0F11103DBB2012B05460B
:101B2000F6D92046FFF7E4FF08212046FFF745FFDE
:101B3000E37E00F0E00203F01F0320461A43082171
:101B4000FFF71FFF29462046BDE8384000F051BC92
:101B500043680BB100211847704700002DE9F0479A
:101B60000446884616461F46FFF78BFF8146002C29
:101B700000F0D7800F2840F0D9802046FFF78DFF76
:101B8000B8F11C0F1AD8DFE808F03F190F2E191909
:101B900037195819979E88198E196119A2A6AAAEED
:101BA00019B2B6191951C400022F00F2018131880F
:101BB000204600F0CEFAB9F10F0F0CD1B8F1100F9A
:101BC00009D06FF085050F21204600F012FC15F1B9
:101BD000860F40F0A8803B46324641462046BDE88D
:101BE000F04701F081BA082F00F2E280D6E9002325
:101BF000204600F0BDFADEE7022F00F2D9803188DE
:101C0000204600F0E6FAD6E7022F06D06FF0150561
:101C1000B9F10F0F40F08780D5E73178A1F10B03C0
:101C20000F2BF3D8204600F0C7FAC4E7022FEDD1FE
:101C30003378002BEAD10225EAE7022F00F2B880C0
:101C4000B6F90010204600F0E1FAF4E7012F00F2A7
:101C5000B2803378013B042BADD801A252F823F0B7
:101C6000751C0008811C0008B71B0008851C0008B3
:101C7000931C00080F21204600F0BBFB012552E019
:101C80001621F8E7A38B5A05F8D52046FFF761FE29
:101C9000F4E72046FFF792FDF0E732782021204656
:101CA00000F02DFB87E7012F00F28280317820467B
:101CB00000F0C1FA0125ABE732784FF4806120468D
:101CC00000F01DFBF6E732784FF40071F7E7327849
:101CD0004FF40051F3E732784FF48041EFE7327868
:101CE0004FF40061EBE732784FF48051E7E7327848
:101CF0004FF48071E3E7012F5AD83178052957D87E
:101D0000A38BDB057FF557AF49B2204600F0AEFA52
:101D1000D0E7012F4CD896F90010204600F0E3FAE6
:101D2000C8E76FF012052846BDE8F087B8F11C0F30
:101D30003FF651AF01A353F828F000BF091C00087B
:101D4000D71B0008A91B0008E71B0008D71B0008C9
:101D5000D71B0008F91B0008D71B00083B1C000814
:101D6000D71B0008B91C0008C71C00089B1C0008F2
:101D7000D71B0008A71C0008D71B00084D1C000833
:101D8000D71B0008CF1C0008D71C0008DF1C000868
:101D9000E71C0008D71B0008EF1C0008F71C000810
:101DA000D71B0008D71B00082D1C0008131D0008B6
:101DB0006FF08A052CE76FF08A05B4E72DE9F04152
:101DC0000446FFF75EFE0F2806464CD00F21204642
:101DD000FFF7F3FD022107462046FFF7EEFD7B07E4
:101DE000054603D5636801212046984738073AD550
:101DF000162E01D0112E08D1A38B590433D5636858
:101E000002212046BDE8F0411847192E01D0122EBC
:101E100029D194F837301BB914490320FEF786FE08
:101E2000013BDBB284F8373023B994F836102046F2
:101E300000F0DFFA6368B3B1A28BD20413D505F0CA
:101E4000E005202D09D002D83DB1BDE8F081602D1C
:101E500007D0A02D03D0BDE8F0810421D1E70521F2
:101E6000CFE70621CDE7BDE8F08100BFAD4F000808
:101E700013B504460121406AFFF7C4F9606AFFF711
:101E80008FFA0121E06AFFF7BDF9E06AFFF791FAE6
:101E90000121206BFFF7B6F9206BFFF781FA0C4B9D
:101EA000009401220021A06AFFF7E6F92046FFF71F
:101EB000F4FD1C212046FFF780FD032805D12046B4
:101EC000FFF77CFC002002B010BD4FF0FF30FAE7B6
:101ED000511B00082DE9F34104460F4690461E466B
:101EE000FFF7ACFD01220DF107012046FFF7B7FD1A
:101EF0009DF8075005F07F05023D1FB92046FFF70A
:101F0000B5FD06E0454508D92046FFF7AFFD6FF067
:101F10006805284602B0BDE8F0812A4639462046C9
:101F2000FFF79DFD022200212046FFF798FD002EBD
:101F3000E4D00122B1182046FFF791FD2046FFF7BB
:101F400095FD07212046FFF738FD3070E1E72DE9C8
:101F5000F04107460D469046FFF7D0FC0026344678
:101F6000464508D1BB8B5B0502D43846FFF7F1FC30
:101F70002046BDE8F0816A68A31C13447F2B05F15D
:101F8000080508D8234655F8081C3846FFF7D1FC49
:101F900001360446E4E76FF08A00BDE8F0810000F6
:101FA00008B5FFF76EFD0F38C0B20A289ABF024B82
:101FB000185C022008BD00BF4F5200082DE9F8430D
:101FC0000F46164698460546002800F09480A1F179
:101FD0000903122B48D8DFE803F017252F4747479E
:101FE000471D4733373B3F47434747470A00B8F150
:101FF000010F40F283800023737000F0E8F8307026
:1020000002242046BDE8F883B8F1010F76D9662393
:102010003380F5E7B8F1000F70D0FFF7C1FF3070E3
:102020000124EEE7838B13F4806F02D00124347017
:10203000E7E700233370F3E7838B13F4007FF4E7C3
:10204000838BC3F34033F5E7838BC3F38033F1E72E
:10205000838BC3F3C023EDE7838BC3F30033E9E73E
:10206000838BC3F30023E5E74346324600F09AFF33
:1020700010F1860F0446C4D12846FFF702FD0F2851
:1020800081463ED12846FFF708FD0E2F1AD008D80A
:10209000012F20D0082F3CD00F21284600F0A9F9AD
:1020A000AFE7182F20D01C2FF6D1B8F1000F33D096
:1020B000284600F00EF90BE0284600F09BF80224B9
:1020C00030802BE0B8F1000F26D0284600F0ACF8A5
:1020D0003070012422E02846FFF7F9FB012408B103
:1020E00034701BE0307019E0B8F1000F14D02846AE
:1020F00000F0B5F8ECE76FF0120482E76FF08A04A5
:102100007FE70E2FDED00ED8012FE4D0082F7FF40A
:1021100078AFB8F1010FCFD86FF08A04B9F10F0F83
:102120007FF46FAFB8E7182FDED01C2FBDD068E763
:1021300038B50A460C4602210546FFF722FC162C4C
:1021400002D185F8344038BD2846FFF79AFC844216
:10215000F6E710B50A0A0446017442742021FFF71D
:1021600010FC227C20462121BDE81040FFF709BC6D
:102170002DE9F843054616461F4600F112080024D3
:102180006FF00709E2003046394601F0DFFB09FB3A
:1021900004F208F8010B38323046394601F0D6FB1C
:1021A00004F12401C2B2C9B228460134FFF7E9FBA9
:1021B000082CE7D1BDE8F883A1F10B020F2A05D85E
:1021C000C27E8A4202D0C176FFF79EBC70470020D3
:1021D000704737B50D0AC181CAB222210446FFF704
:1021E000D0FB2A462321204603B0BDE83040FFF74C
:1021F000C8BB000008B50521FFF7DFFB024B00F06C
:102200000F0033F9100008BD8A520008113109B2DD
:102210001429A8BF142121EAE171024B5A5C05215F
:10222000FFF7AFBB7452000808B52C21FFF7C5FBC0
:10223000C0F3071008BD38B50C462C210546FFF742
:10224000BCFB072C28BF072400F00F0040EA041253
:10225000D2B228462C21BDE83840FFF792BB08B522
:102260002C21FFF7AAFBC0F3420008BD0529A8BF37
:102270000521002938B50C46A8BF0C464FF02C01AB
:102280000546B8BF0724FFF798FB20F00E0040EA90
:102290004402D2B228462C21BDE83840FFF771BB7A
:1022A00038B505460C4699B10A782D21FFF769FB30
:1022B0002E212846FFF781FB637800F0F80203F037
:1022C00007031A4328462E21BDE83840FFF759BBC3
:1022D00038BD08B50921FFF770FB00F00F00400082
:1022E0005B3840B208BD0029C4BF494249B25B31E6
:1022F000C1F3430242F0C0020921FFF742BB10B50F
:10230000838B0446002A40D00B43B1F5807F838342
:102310000AD002D8202929D010BDB1F5007F12D0F3
:10232000B1F5005F29D010BD00F11201FFF7B8FF31
:1023300004212046FFF79AFF53222F212046BDE8B3
:102340001040FFF71EBB2E21FFF737FB40F01002B5
:10235000D2B22E212046FFF714FB17212046FFF7AB
:102360002CFB40F00202D2B21721E7E72E21FFF743
:1023700024FB00F0EF022E21E0E70E21FFF71DFB0A
:1023800040F00402D2B20E21D8E723EA0103B1F5EE
:10239000807F83830AD002D820291CD010BDB1F5DC
:1023A000007F09D0B1F5005F1CD010BD4FF0FF31A8
:1023B000BDE81040FFF75ABF1721FFF7FEFA1721BB
:1023C00000F0FD022046FFF7DCFAA38B9B060FD539
:1023D0002E212046CBE72E21FFF7EFFA40F0100226
:1023E000D2B2C8E70E21FFF7E8FA00F0FB02CAE715
:1023F00010BD38B504460D46FFF743FBA0F11103AD
:10240000DBB2012B1AD91F2818D0A84228D01628D1
:1024100016D1192D03D109212046FFF789FE0F2D72
:1024200018D12046FFF764FB29462046FFF7C5FA7E
:10243000E06AFEF7B5FF84F8345038BD2046DBE78C
:10244000192801D1162DE5E70F28E8D12046FFF71E
:1024500024FBE4E729462046BDE83840FFF768BE84
:1024600038BD10B50446FFF718FB2046FFF709FBFF
:102470001F28FAD02046BDE81040FFF739BB000006
:1024800070B504460D46FDF7E9FF236806463BB9E3
:102490004FF0FF332360FDF7E9FF0125284670BDAB
:1024A000C5B10E4B1D6802212846FDF7DFFE2368EB
:1024B00001330AD105F1080323600023AB603046E5
:1024C000FDF7D4FFFDF7A6FFE7E729462046FEF714
:1024D000AFFBF4E7FDF7CAFFE0E700BFBC02002056
:1024E00070B50446FDF7BAFF256806461DB9BDE87C
:1024F0007040FDF7BBBF6B1C02D100232360F6E7E1
:1025000028460A2150F808392360FDF7AFFE2368FA
:1025100013B94FF0FF33236015F8034C3046FDF735
:10252000A5FF2046BDE87040FDF7E0BE0F4BD3F895
:10253000882042F4700210B5C3F888204FF0006282
:102540009A600B4C102283F822200021DA77601861
:102550000131522980F80023F9D11A6942F01002A2
:102560001A615A6942F400725A6110BD00ED00E030
:1025700000E100E0F0B58468A68BE3898FB006F037
:102580002800ADF8183040F001000D4621B96FF079
:10259000150420460FB0F0BD91F91030013341D140
:1025A00089680B790A7813F0C00F05BF02F10803A0
:1025B0004F781F4B5B1818BF022752B3083194F8AD
:1025C0001AE00EF10106A676039008AEBDF81800D9
:1025D000ADF80800ADF804000097CDF810E03046E3
:1025E00000F0B6FB07460028D1D0284607A900F026
:1025F0006BFB0546C8B181682368079A1B6881E8B0
:10260000C0002046984700210446284600F04EFBB3
:10261000BFE7720747BF04F11201082204F110015D
:102620000222CCE76FF04C04B3E76FF06804B0E728
:10263000D15200082DE9F04387683B685C680023AD
:1026400087B01A4619463846A047041E04DC002409
:10265000204607B0BDE8F0830023224619461846FD
:1026600000F032FA06460028F1D03B6881685D68C8
:1026700022466B463846A847B0F1000804DC00212A
:10268000304600F013FBE2E7BA8B12F0020557D197
:10269000B06800F0DFFB044620B92146304600F068
:1026A00005FBD5E70146A8EB00082A46304600F0B6
:1026B00025FA04460028F0D0856801AA04A9284616
:1026C00000F03AFC01AA814602A9284600F0E4FB8A
:1026D000B9F1000FD3DB0028D1DBC1B25FFA89F377
:1026E00004AA02A800F0E4F805460028C7D0B9F112
:1026F000020F0CD19DF81030FF2B08D19DF811303E
:10270000FF2B04D18268137963F07F031371AB68E8
:102710009DF801209A719DF800205A710B4A128889
:102720005A803B7B33742146304600F0F9FA00238F
:102730006B60334600E013465A68002AFBD15D60A7
:102740004146304600F046FA344681E7B8020020A0
:10275000034B0360034B436081600020704700BF60
:102760007525000835260008F0B5254E84683388A5
:10277000838195B00821054604A801F083F83088CC
:10278000204B6360A56000B200F084F82368204607
:102790009B68984741F2342740F20326684601F0CF
:1027A0006DF8BDF80230B34213D0B3F5017F08D203
:1027B00040F202229342F1D12B68019928469847B2
:1027C000EAE718D0BB42E9D123682046DB68984786
:1027D000E2E7236801995E690B894A680978204617
:1027E000B04740F20523039002A96846ADF80A30CD
:1027F00001F016F8D0E7236801991E69ECE700BFE5
:10280000B80200200928000813B5806881B941F298
:1028100034230190B0F90C10ADF80230684600F096
:10282000B9FF002802DC0D4801F0D4FB02B010BD56
:102830000229FBD14368984704460028F6D0034696
:10284000074990F9100040F2012201F02FF80146EB
:102850000028EBD1204600F029FAE7E7AA52000849
:102860000000FFFF30B585B0089C74B1A56865B164
:102870000293074B009301940823FEF7F9F900280F
:10288000D8BF6FF0150005B030BD6FF01200FAE749
:1028900069270008054AB2F90030984204D013B104
:1028A0006FF00B007047108000207047E00F002091
:1028B0002DE9F041174603F108020A440E460021B3
:1028C00080461C4608464FF0FF3300F0FDF80546F1
:1028D000E8B18068002306704470438043718371BF
:1028E0000371B8F1000F05D026B1324641460830D9
:1028F00001F0E9FA5FB154B1A8684378A34206D168
:102900000378083322463946184401F0DCFA284699
:10291000BDE8F08170B503461A4A072B88BF033320
:1029200010688CBF23F003030823002140B34468E0
:10293000A34210D8E41A072C0344134E0ED9C6F153
:1029400008051D44B5F5C05F15D900211160026866
:1029500083E8140005E001460068E7E7046841B930
:1029600014600A4A9B1B11889BB2994208D21380BB
:1029700070BD0C60F5E709B91360E8E70B60E6E7A6
:1029800070BD00BFE40F0020EC0F0020EC270020FA
:1029900008B502490320FEF7C9F800BFAD4F000893
:1029A00001210148FFF76CBDE80F002038B51E4B30
:1029B000C31AB3F5C05F36D21C4C226800230AB19B
:1029C000824211D307298ABF0331082121F0030174
:1029D000174D02604218AA1A072A98BF8918416049
:1029E0002BB92060034611E013461268E7E75A68E6
:1029F00018601A44821A072AF4D808B9FFF7C8FFEA
:102A000002681A604268C11A0A445A601A6852B1D0
:102A100059681944511A072905D811681960D11A43
:102A200052680A445A6038BDEC0F0020E40F0020C1
:102A3000EC2700202DE9F843814614200F46164666
:102A40009846FFF767FF044650B166B13046FFF77E
:102A500061FF054640B920461421FFF7A7FF2C4629
:102A60002046BDE8F88335460123C4F80490A560EC
:102A7000E66084F810802360002FF1D0324639469A
:102A8000284601F020FAEBE7F8B50E4D0446002683
:102A900004B9F8BD631BB3F5C05F01D3FFF778FF3E
:102AA00094E88800012B0AD1E168A0682660FFF74E
:102AB0007DFF14212046FFF779FF3C46E8E7013B04
:102AC0002360FAE7EC0F0020B2F5C05FF8B50546C9
:102AD0000E4614461F460DD8FFF762FF22463B46BE
:102AE00031462846FFF7A6FF04460348FFF7F8FCE7
:102AF0002046F8BD0024FBE7E80F002007292DE958
:102B0000F84388BFCF1C0D468CBF27F0030708276A
:102B100004469146FFF744FF2DB124B1E3689D427E
:102B200001D8A36833B92A48FFF7DAFC00263046FB
:102B3000BDE8F8831420FFF7EDFE06460028F2D02A
:102B4000E3689D423DD0AF4202D85A1B072A38D8CD
:102B50002846FFF7DFFE074620B914213046FFF76D
:102B600025FFE0E7E068401BFFF7D4FE804630B960
:102B700014213046FFF71AFF29463846EFE72A4668
:102B8000A168384601F09FF9E268A168521B294408
:102B9000404601F098F9E168A068FFF707FFC4F824
:102BA0000880E3680A485B1BE36063687360012385
:102BB000B760F56086F8109033606660FFF790FCB0
:102BC000B5E7A7689D4214BF7B190023A360E8E71F
:102BD000E80F0020072970B588BFCE1C04468CBFC3
:102BE00026F0030608260D46FFF7DAFE1CB9234936
:102BF0000320FDF79BFFE368A06843B90028F6D1E6
:102C00009D420CD11E48FFF76BFC002070BD0028D0
:102C1000EDD01C4A821AB2F5C05FF1D3E7E735B9AF
:102C200038B11946FFF7C2FEA560E560EAE79D42AC
:102C300002D8991B072917D82846FFF76BFE0646CE
:102C400020B90F48FFF74CFC0C2070BDA16829B1DA
:102C5000E268AA4228BF2A4601F035F9E168A06877
:102C6000FFF7A4FEA660E0E7033323F003039E42D0
:102C7000DBD23044FFF79AFED7E700BFAD4F000824
:102C8000E80F0020EC0F002038B504460D46FFF792
:102C900087FE24B90448BDE83840FFF721BC23680B
:102CA0002B4423606468F4E7E80F002010B5044665
:102CB000FFF776FE2046FFF7E7FE0248BDE810402A
:102CC000FFF70EBCE80F002070B504460E4619B998
:102CD00012490320FDF72AFF10B90020306070BDB3
:102CE00001460025496801350029FBD16FF0010339
:102CF000EA002046FFF7E8FE0028EED08368002BAC
:102D0000E6D00833A26843F8082CE268646843F808
:102D1000042C0833002CF5D1356070BDAD4F000890
:102D200010B504468C42084606D164680021416013
:102D3000FFF7BCFF204610BD23465A68002AF5D095
:102D4000904202D142685A60F0E71346F5E700006E
:102D5000F8B504460F461E4610219DF8243006980B
:102D600023706170154602B1B7B100B1A6B113F07E
:102D7000050F02D00DB9002869D09DF82830A37046
:102D8000002861D09DF82030E37002289DF82130A2
:102D9000237103D0082827D00020F8BD02462C4913
:102DA000304601F081F818B9237823F0200323700E
:102DB000637843F008036370737863713378A371A9
:102DC0000720002D43D0BDF81C20BDF820309A42CA
:102DD00017D1237843F040032370022D1AD0082D19
:102DE00023D0002DD8D1F8BD1C236370221D06F11D
:102DF000080313F8011D02F8011FB342F9D10D2099
:102E0000DFE7431C9DF81C2022549DF81D20E2544E
:102E10000230E2E7637863F07F0363707A782254CC
:102E2000431C3A78E2540230F8BD637863F03F0304
:102E3000637007F10803044413F8012D04F8012B13
:102E4000BB42F9D10830F8BD0320002DD9D1F8BD1F
:102E5000D1520008427802F00C03082B014611D031
:102E60000C2B11D0B3B90078400613D4032012F014
:102E7000C00210D00B785B0658BF0230802A05D103
:102E8000023070470720F2E70D20F0E7C02A01D199
:102E9000083070470020704770B501B11AB9254954
:102EA0000320FDF743FE437803F00C03082B08D101
:102EB00003785C0603D5C378137003795370072336
:102EC00012E00C2B08D103785B0603D5C37813708E
:102ED000037953700D2307E013B16FF0150070BD37
:102EE00003785E06F9D40323447814F0C00411D0AB
:102EF00005786D0605D4C65C16705D1C0233455D11
:102F00005570802C08D1C25C4A70184443780B700D
:102F1000022070BD204670BDC02CDED1184401F1E6
:102F2000080310F8012B03F8012D9942F9D108206C
:102F300070BD00BFAD4F000808B501B11AB91849FE
:102F40000320FDF7F3FD437803F00C03082B09D1B0
:102F5000C37813700379537043794B7083790B7086
:102F6000022008BD0C2B0ED1C378137010F8043F5B
:102F7000537001F1080310F8012F03F8012D8B4263
:102F8000F9D1082008BD3BB9037813F0400F14BFF6
:102F90006FF01500002008BD6FF0150008BD00BFE0
:102FA000AD4F000810B5044610461A2900F296806D
:102FB000DFE801F033940E1C25252F55949494944A
:102FC0009439944B9445949494949494949451008B
:102FD000012B03D843490320FDF7A8FD022204F189
:102FE000100100F070FF0223184610BD072BF1D925
:102FF000082204F1120100F066FF0823F4E7022B17
:10300000E8D1A28B520702D508220280ECE70380A8
:10301000EAE7022BDED1E289F7E7022BDAD1E37E81
:1030200003800123E0E7012BD4D1A38B13F0200F01
:1030300002D001230370D7E700230370F1E7012BCF
:10304000C8D1A38B13F0020FF2E7012BC2D194F980
:103050000C200270C8E7022BBCD10322D5E7072B56
:10306000B8D9A38B5B074CBF082302234FF00002A3
:103070004CBF04F1120104F11001042B42700270E4
:1030800018D0082B03D0022BB7D1134619E00A78C9
:1030900082F0020202704A7842708A788270CA789E
:1030A000C2700A7902714A7942718A798271CA7949
:1030B000C27199E70B7883F0020303704B78437079
:1030C0000223FF240022C470FE2482700471427126
:1030D000CA5C827119444B78C3718EE76FF0850327
:1030E00082E700BFAD4F000870B515461C46112998
:1030F00064D8DFE801F0096315253535456363635E
:103100006363634A635D6354022C03D02D4903203B
:10311000FDF70CFD1388FF2BF8D8C376204670BD51
:10312000022CF3D800F1100602220021304600F0F4
:10313000D5FE22462946304600F0C5FE0224EDE7C2
:10314000082CE3D800F1120608220021304600F0D6
:10315000C5FE22462946304600F0B5FE0824DDE7CC
:10316000022CD3D11388022B05D0082BD6D1838B08
:1031700043F0040302E0838B23F004038383CDE751
:10318000022CC3D11388C381C8E71278838B1AB18C
:1031900043F020038383D1E723F02003FAE712787A
:1031A000838B12B143F00203F4E723F00203F1E74B
:1031B000012CABD192F900300373AFE76FF08504B7
:1031C000ACE700BFAD4F00088368DB0710B50446CD
:1031D00006D5C068064BC0B253F821309847E0606E
:1031E000044B1B681BB1BDE81040FDF707BD10BDC7
:1031F000F8270020C00200202DE9F04F8BB020B14D
:1032000001286FD04FF0FF3069E03D4A019205235D
:1032100007210292039204930793059108930622D3
:103220000692099300210DF104080DF1100C4FF0E6
:10323000030E0227012607AC5CF8212058F8213044
:103240005000D3F800B00EFA00FA6FEA0A090BEA50
:10325000090BC3F800B0D3F800B007FA00F04BEA4E
:10326000000BC3F800B0D3F808B009EA0B0BC3F8A1
:1032700008B0D3F808B04AEA0B0AC3F808A0D3F89C
:1032800004A006FA02FB2AEA0B0AC3F804A0D3F84A
:103290000CA009EA0A09C3F80C90D3F80C90072A8D
:1032A00040EA0900D4BF4FF000094FF00109D8608F
:1032B00003EB8903A2EBC902186A92000F2505FAF5
:1032C00002F920EA0900186254F82150186A05FA38
:1032D00002F20131024303291A62ADD100200BB082
:1032E000BDE8F08F0D23074A04930F2105230192B7
:1032F000029203920793059108930E2290E700BF74
:103300000000024000040240F8B506460F46042AB9
:1033100004D8DFE802F00D06101418004FF0FF305B
:10332000F8BD2C4B1C5C0534E4B286B1012E3ED0B6
:103330006FF00100F8BD274B1C5C0434F4E7254B0B
:103340001C5C0234F0E7234B1C5C0134ECE74FF4C7
:1033500080510120FEF7DEF801210220FEF7DAF8A5
:1033600001210220FEF7D6F801210220FEF7D2F853
:10337000194D3046FFF740FFEB69002023F400634E
:10338000EB61286068602B6843F440732B602B6806
:1033900043EAC4042C602B6843F004032B602B68C1
:1033A0001F432F602B6843F040032B60F8BD4FF4A0
:1033B00080410020FEF7AEF802210846FEF7AAF889
:1033C00002210846FEF7A6F802210846FEF7A2F8F9
:1033D000024DCEE7D35200080030014000380040D3
:1033E000012808B507D8054B012103EB8000FFF742
:1033F00047F8002008BD4FF0FF3008BDF02700203F
:10340000012808B506D8054B03EB8000FFF768F8E4
:10341000002008BD4FF0FF3008BD00BFF02700209E
:1034200070B101280ED1094B98688007FCD5D9608E
:103430009968C907FCD5DB6802B113700120704799
:10344000034BF1E74FF0FF30704700BF00380040FA
:103450000030014000210148FFF7B6BE00300140B6
:1034600001210148FFF7B0BE003800402DE9F341CB
:1034700006460D46174698460024444503D120468B
:1034800002B0BDE8F0810DF107025DB1295D304663
:10349000FFF7C6FF002807DB17B19DF807303B5543
:1034A0000134EAE72946F2E74FF0FF30E8E770B56C
:1034B00016461A4605461C46FFF7B2FF002802DAF8
:1034C0004FF0FF3070BD224631462846FFF7A8FF77
:1034D0000028F5DB012070BD0C22014900F0F3BC8F
:1034E000107AFF1FFEF7FCBF38B504460020FEF738
:1034F00083F805460020FEF77FF8401BA042F9D371
:1035000038BD000030B587B004460D46FCF7B1FF6A
:1035100048B11DB10E490320FDF708FB2046FFF717
:10352000E3FF07B030BD0B4B0090039002900121E8
:1035300068460493CDF814D0FEF7A2FF214601A8F7
:103540002A46FDF7A3FA01216846FEF799FFE8E74E
:10355000AD4F0008E5340008F8B505460E46FCF707
:103560007DFF364B364A1B881BB2074652F8233084
:103570001A6A002A4ED05C699969A1424AD9611C35
:103580005961D9690C4046B9196931B9611C04D136
:103590003846FCF76BFF2046F8BD002C3EDB02EB03
:1035A000C40103C985E803001E69002E38D03168C4
:1035B0001961002C1EDA736893E8030085E80300A4
:1035C00016F8043C052B23D0002373600A21A6F1D2
:1035D0000800FCF74BFE16F8034C3846FCF746FF94
:1035E0000E2C28D82046FCF781FE24E03846FCF754
:1035F0003DFF20E09D695969D869691A8842A9BFD1
:10360000691C4FF0FF350540996102EBC505D2E713
:103610000F24E2E74FF0FF34002EB5D0DD60C3E7A2
:10362000002CE3DA18460321FCF720FE3846FCF7AD
:103630001DFFFCF7EFFE0124ADE700BFB80200203C
:103640000803002010B583694469C2691C1BA242AB
:1036500001DA002010BD5C1C13408461F9D4026AB9
:1036600003C902EBC30383E80300012010BD00007F
:103670002DE9F8431E46264B53F82150254B1B8855
:103680000380074691463DB93046FCF7EFFE4FF008
:10369000FF342046BDE8F8832B79032B2ED01E4B38
:1036A00001462846D3F80080FFF7CCFF044650B10E
:1036B0003046FCF7DBFE98F80430052B01D1FCF70F
:1036C000A9FE0124E5E7B9F1000F03D13046FCF76C
:1036D000CDFEDEE798F80430C8F80C70052B0CBF5F
:1036E000052104214046FCF7C1FD414605F11000CB
:1036F000FDF79EFA3046FCF7B9FEE0E703C8EB6839
:1037000083E803000A212846FCF7B0FDF2E700BF7A
:1037100008030020B8020020BC02002038B504468F
:10372000FCF79CFE074B1B882380074B2146054670
:103730001868FFF787FF04462846FCF797FE2046E7
:1037400038BD00BFB8020020BC02002008B50F4BF6
:1037500053F82130B3B1212202801A79032A0BD108
:1037600003C8DA6882E8030018460A21FCF77EFDE8
:10377000074B0120186008BD01461846BDE8084007
:10378000FFF760BF4FF0FF3008BD00BF0803002007
:10379000C002002070B504460D46FCF76AFE28B151
:1037A00029462046BDE87040FFF7D0BF094B1B8873
:1037B0001BB29D4204D12046BDE87040FFF7AEBF6A
:1037C000FCF74CFE2946034601222046BDE8704026
:1037D000FFF74EBFB802002070B504460D46FCF757
:1037E00048FE064628B129462046BDE87040FFF74E
:1037F000ADBF0A4B1B881BB29D4204D12046BDE8D9
:103800007040FFF78BBFFCF729FE3246034629467E
:103810002046BDE87040FFF72BBF00BFB802002074
:1038200070B504460D46FCF719FEB4F90020114BA3
:1038300053F8224006461CB90F490320FDF776F9DC
:103840002379052B04D0FCF711FE4FF0FF3070BD3B
:1038500095E80300E36883E803000A212046FCF7AB
:1038600005FD64793046FCF701FE2046FCF73EFD7D
:10387000012070BD08030020AD4F00080121FFF7B3
:103880006BBE000008B5074B4A1E1B68114018624A
:1038900003D005490320FDF749F959619961DA61BF
:1038A00008BD00BFBC020020AD4F00082DE9F34168
:1038B0000446884617461E4600F032F8054648B1D1
:1038C0004146204600F01EF8691E04463046FFF7C8
:1038D000DBF91CB9284602B0BDE8F081B4F9081044
:1038E000ADF8027068460196FFF776FF002803DC0A
:1038F00000213046FFF7DAF9204600F01FF80446B1
:10390000E7E7000040B9054B186800B97047436805
:103910008B4202D00068F8E70020704700280020A2
:1039200040B9054B1B6803B970475A688A4208BF03
:103930000130F7E7002070470028002028B14368D5
:10394000006810B142689342FAD17047D0400B1C16
:10395000D1409C46203AD34018435242634693409C
:103960001843704780F0004002E000BF81F0004142
:1039700042001FBF5FEA410392EA030F7FEA226C15
:103980007FEA236C6AD04FEA1262D2EB1363C1BFA5
:10399000D218414048404140B8BF5B42192B88BF14
:1039A000704710F0004F40F4000020F07F4018BF37
:1039B000404211F0004F41F4000121F07F4118BF57
:1039C000494292EA030F3FD0A2F1010241FA03FCFF
:1039D00010EB0C00C3F1200301FA03F100F00043E7
:1039E00002D5494260EB4000B0F5000F13D3B0F1AF
:1039F000807F06D340084FEA310102F10102FE2A1E
:103A000051D2B1F1004F40EBC25008BF20F001008D
:103A100040EA03007047490040EB000010F4000F3B
:103A2000A2F10102EDD1B0FA80FCACF1080CB2EBCE
:103A30000C0200FA0CF0AABF00EBC250524218432D
:103A4000BCBFD0401843704792F0000F81F40001D2
:103A500006BF80F400000132013BB5E74FEA4103A5
:103A60007FEA226C18BF7FEA236C21D092EA030F11
:103A700004D092F0000F08BF0846704790EA010F8B
:103A80001CBF0020704712F07F4F04D1400028BFB8
:103A900040F00040704712F100723CBF00F500009A
:103AA000704700F0004343F0FE4040F400007047D0
:103AB0007FEA226216BF08467FEA2363014642027C
:103AC00006BF5FEA412390EA010F40F4800070478F
:103AD0004FF0000304E000BF10F0004348BF404235
:103AE0005FEA000C08BF704743F0964301464FF071
:103AF00000001CE050EA010208BF70474FF00003CD
:103B00000AE000BF50EA010208BF704711F000430D
:103B100002D5404261EB41015FEA010C02BF8446DD
:103B20000146002043F0B64308BFA3F18053A3F53C
:103B30000003BCFA8CF2083AA3EBC25310DB01FA83
:103B400002FC634400FA02FCC2F12002BCF1004F07
:103B500020FA02F243EB020008BF20F00100704798
:103B600002F1200201FA02FCC2F1200250EA4C00EC
:103B700021FA02F243EB020008BF20EADC70704732
:103B80004FF0FF0C1CEAD0521EBF1CEAD15392EA40
:103B90000C0F93EA0C0F6FD01A4480EA010C40021C
:103BA00018BF5FEA41211ED04FF0006343EA501076
:103BB00043EA5111A0FB01310CF00040B1F5000FB8
:103BC0003EBF490041EAD3715B0040EA010062F167
:103BD0007F02FD2A1DD8B3F1004F40EBC25008BF51
:103BE00020F00100704790F0000F0CF0004C08BF6F
:103BF00049024CEA502040EA51207F3AC2BFD2F13C
:103C0000FF0340EAC250704740F400004FF0000349
:103C1000013A5DDC12F1190FDCBF00F00040704783
:103C2000C2F10002410021FA02F1C2F1200200FAC1
:103C300002FC5FEA310040F1000053EA4C0308BF88
:103C400020EADC70704792F0000F00F0004C02BFD9
:103C5000400010F4000F013AF9D040EA0C0093F054
:103C6000000F01F0004C02BF490011F4000F013BAE
:103C7000F9D041EA0C018FE70CEAD15392EA0C0F1C
:103C800018BF93EA0C0F0AD030F0004C18BF31F087
:103C9000004CD8D180EA010000F00040704790F05D
:103CA000000F17BF90F0004F084691F0000F91F001
:103CB000004F14D092EA0C0F01D142020FD193EAC7
:103CC0000C0F03D14B0218BF084608D180EA01004F
:103CD00000F0004040F0FE4040F40000704740F02B
:103CE000FE4040F4400070474FF0FF0C1CEAD052F9
:103CF0001EBF1CEAD15392EA0C0F93EA0C0F69D055
:103D0000A2EB030280EA010C49024FEA402037D0BF
:103D10004FF0805343EA111143EA10130CF00040B6
:103D20008B4238BF5B0042F17D024FF4000C8B42A6
:103D300024BF5B1A40EA0C00B3EB510F24BFA3EB86
:103D4000510340EA5C00B3EB910F24BFA3EB910356
:103D500040EA9C00B3EBD10F24BFA3EBD10340EAB0
:103D6000DC001B0118BF5FEA1C1CE0D1FD2A3FF6F6
:103D700050AF8B4240EBC25008BF20F001007047AB
:103D80000CF0004C4CEA50207F32C2BFD2F1FF034E
:103D900040EAC250704740F400004FF00003013A7F
:103DA00037E792F0000F00F0004C02BF400010F423
:103DB000000F013AF9D040EA0C0093F0000F01F037
:103DC000004C02BF490011F4000F013BF9D041EA59
:103DD0000C0195E70CEAD15392EA0C0F08D142028C
:103DE0007FF47DAF93EA0C0F7FF470AF084676E75F
:103DF00093EA0C0F04D14B023FF44CAF08466EE738
:103E000030F0004C18BF31F0004CCAD130F0004205
:103E10007FF45CAF31F000437FF43CAF5FE700BF5D
:103E200042000ED2B2F1FE4F0BD34FF09E03B3EB24
:103E3000126209D44FEA002343F0004323FA02F050
:103E400070474FF00000704712F1610F01D142023C
:103E500002D14FF0FF3070474FF00000704700BFB5
:103E600070B50D4E0D4CA41BA4100025A54209D120
:103E70000B4E0C4CFCF788F9A41BA4100025A5429E
:103E800005D170BD56F8253098470135EEE756F854
:103E9000253098470135F2E7705300087053000849
:103EA000705300087053000810B501390244904265
:103EB00001D1002010BD10F8013B11F8014FA342C1
:103EC000F5D0181B10BD10B5431E0A44914200D115
:103ED00010BD11F8014B03F8014FF7E70244034608
:103EE000934200D1704703F8011BF9E70FB40A4B66
:103EF00013B51C6824B1A36913B9204600F024FA55
:103F000005AB049AA1680193204600F0DBFB02B0E8
:103F1000BDE8104004B070475002002070B50E4656
:103F2000054618B183690BB900F00EFAAB69AC68AD
:103F300013B9284600F008FA234B9C4217D16C684D
:103F4000A3891B071DD52369DBB1013EA36816F8C1
:103F5000011F013BA360E9B9002B2EDA22460A219A
:103F6000284600F03FF8013011D00A2070BD174BF1
:103F70009C4201D1AC68E3E7154B9C4208BFEC685A
:103F8000DEE72146284600F07FF80028DDD04FF01C
:103F9000FF3070BD002B04DAA269934206DB0A29C8
:103FA00004D023685A1C22601970CFE722462846A5
:103FB00000F018F80130C9D1E9E723680A205A1C3B
:103FC0002260187070BD00BFFC5200081C5300082E
:103FD000DC520008024B01461868FFF79FBF00BF84
:103FE00050020020F8B50E461446054618B1836904
:103FF0000BB900F0A9F9214B9C422AD16C68A36946
:10400000A360A3891A072ED5236963B323692068A7
:10401000C01A6369F6B29842374604DB2146284647
:1040200000F028F928BBA368013BA36023685A1C51
:1040300022601E7063690130984204D0A389DB07B7
:1040400019D50A2E17D12146284600F013F990B150
:104050000FE00B4B9C4201D1AC68D0E7094B9C426E
:1040600008BFEC68CBE72146284600F00DF8002891
:10407000CCD04FF0FF373846F8BD00BFFC520008E7
:104080001C530008DC520008324B70B51D68064610
:104090000C4625B1AB6913B9284600F055F92E4BF3
:1040A0009C420FD16C68B4F90C309AB215072CD42D
:1040B000D00611D40922326043F04003A3814FF0AF
:1040C000FF3070BD254B9C4201D1AC68EBE7244B1F
:1040D0009C4208BFEC68E6E7510712D5616B41B11D
:1040E00004F14403994202D0304600F017FA00234D
:1040F0006363A38923F02403A381002363602369FE
:104100002360A38943F00803A38123694BB9A389E2
:1041100003F42073B3F5007F03D02146304600F04E
:10412000C1F9A28912F001030CD00023A3606369D6
:104130005B42A361236953B9B4F90C3013F08000DA
:10414000BAD170BD920758BF6369A360F2E700203F
:10415000F7E700BF50020020FC5200081C53000883
:10416000DC5200088A892DE9F041054610070C460B
:104170005AD44B68002B05DC0B6C002B02DC0020B2
:10418000BDE8F081E66A002EF9D0002312F48052D7
:104190002F682B6033D0606DA3895A0705D56368FB
:1041A000C01A636B0BB1236CC01A00230246E66A87
:1041B000216A2846B047431CA38906D129681D29D6
:1041C0004BD82B4ACA40D60747D500226260D90493
:1041D0002269226004D5421C01D12B6803B96065B5
:1041E000616B2F600029CAD004F14403994202D0C8
:1041F000284600F093F900206063BDE8F081216A51
:1042000001232846B047411CC6D12B68002BC3D0E0
:104210001D2B01D0162B01D12F60B0E7A38943F0ED
:104220004003A381BDE8F0810F69002FA7D0930759
:104230000E6808BF4B690F6018BF0023A6EB070884
:104240008B60B8F1000F9ADD43463A46216AA66AB0
:104250002846B047002807DCA38943F04003A38128
:104260004FF0FF30BDE8F0810744A8EB0008E8E715
:104270000100402038B50B6905460C46DBB118B18A
:1042800083690BB900F060F80C4B9C4209D16C6853
:10429000B4F90C307BB121462846BDE83840FFF721
:1042A00061BF074B9C4201D1AC68F1E7054B9C42D2
:1042B00008BFEC68ECE7002038BD00BFFC520008E6
:1042C0001C530008DC520008014900F0A9B800BFE7
:1042D00075420008002310B5044603604360836004
:1042E00081814366C281036143618361194608226B
:1042F0005C30FFF7F3FD054B6362054BA362054B92
:10430000E362054B2462236310BD00BF1D4C00080F
:104310003F4C0008774C00089B4C000870B54A1EC3
:10432000682555430E4605F1740100F045F9044631
:1043300040B1002180E842000C30A06005F1680225
:10434000FFF7CCFD204670BD836910B5044633BB32
:104350008364C3640365124B124A1B6882629842ED
:1043600004BF0123836100F01FF86060204600F065
:104370001BF8A060204600F017F80022E06004213E
:104380006068FFF7A7FF01220921A068FFF7A2FFDD
:1043900002221221E068FFF79DFF0123A36110BDF7
:1043A000D8520008C9420008F8B51C4B1E68B36912
:1043B000074613B93046FFF7C7FF4836B46873683D
:1043C000013B03D5336833B13668F7E7B4F90C50D5
:1043D0006DB16834F4E704213846FFF79FFF306081
:1043E0000028F1D10C233B6004462046F8BD4FF66F
:1043F000FF73E3810123A38165662560A560656085
:1044000025616561A5610822294604F15C00FFF77A
:1044100065FD6563A563A564E564E6E7D852000819
:104420002DE9F8438046894600F14804002614B976
:104430003046BDE8F883A5686768013F01D5246868
:10444000F5E7AB89012B07D9B5F90E30013303D05D
:1044500029464046C84706436835EEE770B50E4624
:10446000B1F90E10002990B014461D4607DA00235A
:104470002B60B3891A0610D44FF480630EE001AAB2
:10448000FBF7B6FE0028F2DB029A02F47042A2F5B6
:1044900000535A425A412A60EEE74023002023602D
:1044A00010B070BD8B8973B59D0706460C4607D5C5
:1044B00004F14703236023610123636102B070BDEF
:1044C00001AB6A46FFF7CAFF00990546304600F087
:1044D00073F838B9B4F90C309A05EFD443F00203FD
:1044E000A381E5E70C4BB362A389206043F080030E
:1044F000A381009B6361019B20614BB1B4F90E1055
:104500003046FBF77AFE18B1A38943F00103A3817B
:10451000A3891D43A581D1E7C942000838B50546E6
:10452000002945D051F8043C0C1F002BB8BFE418FB
:1045300000F00EFC1F4A1368104633B96360146024
:104540002846BDE8384000F004BCA3420CD92168DD
:104550006218934204BF1A685B68636004BF521814
:1045600022600460ECE713465A680AB1A242FAD905
:1045700019685818A0420BD120680144581882428B
:104580001960DDD1106852685A6001441960D7E79C
:1045900002D90C232B60D3E7206821188A4204BF7C
:1045A00011685268626004BF091821605C60C7E747
:1045B00038BD00BF0428002070B5CD1C25F00305D0
:1045C00008350C2D38BF0C25002D064601DBA9420D
:1045D00003D90C233360002070BD00F0B9FB234ADF
:1045E0001468214691B9224C23681BB93046FBF769
:1045F000CFFD206029463046FBF7CAFD431C26D17B
:104600000C233360304600F0A4FBE4E70B685B1B2F
:104610001AD40B2B0FD90B60CD50CC18304600F0BC
:1046200098FB04F10B00231D20F00700C31A1BD0D8
:104630005A42E25070BD8C420DBF63684B686360A4
:10464000136018BF0C46E9E70C464968CAE7C41C6A
:1046500024F00304A04205D0211A3046FBF798FD50
:104660000130CDD02560D9E770BD00BF04280020FF
:10467000082800209368013B002B10B4936008DAEF
:104680009469A34202DBCBB20A2B02D110BCFFF724
:10469000A9BC1368581C10601970C8B210BC7047D0
:1046A000F8B506460F461446D518AC4201D1002095
:1046B00007E03A4614F8011B3046FFF7DBFF431CC6
:1046C000F3D1F8BD2DE9F04F9DB00C46174603938A
:1046D000064618B183690BB9FFF736FE7C4B9C4246
:1046E00057D17468A38918075DD52369002B5AD068
:1046F0000023099320238DF8293030238DF82A30A8
:104700004FF0010BB846454615F8013B002B55D13B
:10471000B8EB070A0BD053463A4621463046FFF71E
:10472000BFFF013000F0C480099B5344099398F8FF
:104730000030002B00F0BC8000234FF0FF320493C8
:104740000793059206938DF853301A930522297822
:10475000604800F0ADFA05F10108049B002831D152
:10476000D90644BF20228DF853201A0744BF2B22BC
:104770008DF853202A782A2A2CD0079A00210A2063
:10478000A846013598F80030303B092B6DD971B33C
:1047900026E0514B9C4201D1B468A3E74F4B9C42A9
:1047A00008BFF4689EE721463046FFF76DFC0028FD
:1047B0009ED04FF0FF301DB0BDE8F08F252BA7D065
:1047C000A846A0E7434A801A0BFA00F01843049069
:1047D0004546BBE7039A111D12680391002A01DBCD
:1047E000079204E0524243F002030792049398F8C0
:1047F00000302E2B10D198F801302A2B08F101013E
:1048000037D1039B1A1D1B680392002BB8BF4FF0D2
:10481000FF3308F102080593314D98F80010032288
:10482000284600F045FA40B14023401B03FA00F04F
:10483000049B0343049308F1010898F800102948E9
:104840008DF82810062208F1010700F031FA00283F
:1048500034D0254B03BB039B073323F007030833F6
:104860000393099B4B4409934CE700FB023201215F
:1048700086E70023059318460A258846013198F8F3
:104880000020303A092A03D9002BC5D00590C3E790
:1048900005FB00200123F0E703AB00932246134BF6
:1048A00004A93046AFF30080B0F1FF3F8146D8D174
:1048B000A3895B063FF57DAF09987CE703AB0093C6
:1048C00022460A4B04A9304600F088F8ECE700BF06
:1048D000FC5200083C5300081C530008DC5200083E
:1048E000425300084653000800000000A14600089B
:1048F0002DE9F04791461F468A680B69DDF8208054
:104900009342B8BF1346C9F8003091F843200646D9
:104910000C4612B10133C9F800302368990642BF32
:10492000D9F800300233C9F80030256815F00605C3
:1049300007D104F1190AE368D9F800209B1A9D42B7
:1049400029DB94F843302268003318BF0123920614
:104950002ED404F1430239463046C047013021D0FD
:104960002368E568D9F8002003F00603042B08BF8C
:10497000AD1AA36822690CBF25EAE57500259342AC
:10498000C4BF9B1AED184FF000091A344D451BD1D6
:104990000020BDE8F0870123524639463046C04723
:1049A000013003D14FF0FF30BDE8F0870135C2E799
:1049B000E1185A1C302081F84300224494F8451035
:1049C00082F843100233C4E70123224639463046B9
:1049D000C0470130E6D009F10109D7E72DE9F043DE
:1049E00017460A7E85B06E2A984606460C460C9BF2
:1049F00001F1430E00F0BC801AD8632A2ED00AD8E9
:104A0000002A00F0C880582A00F08A8004F142058C
:104A100084F842202AE0642A01D0692AF6D121686C
:104A20001A6811F0800F23D0111D1960136827E058
:104A3000732A00F0B48008D86F2A2AD0702AE5D1F2
:104A40000A6842F020020A6003E0752A21D0782A21
:104A5000DCD1782284F845206E4964E01A6801F1BF
:104A60004205111D1960136884F842300123A3E048
:104A700011F0400F02F104011960D7D0B2F90030F3
:104A8000002B03DA2D225B4284F8432062490A227C
:104A900017E02068196810F0800F03D0081D186017
:104AA0000B6806E010F0400F01F104001860F7D029
:104AB0000B8859496F2A14BF0A220822002084F863
:104AC00043006568A560002DC0F29C80206820F03E
:104AD00004002060002B3FD1002D40F095807546EA
:104AE000082A0BD12368DA0708D5236962689A423D
:104AF000DEBF302305F8013C05F1FF35AEEB0503C1
:104B00002361CDF800803B4603AA21463046FFF7DB
:104B1000EFFE013055D14FF0FF3005B0BDE8F08316
:104B200081F845203C492268186812F0800F00F196
:104B300004051D6001D0036802E05506FBD503881B
:104B4000D00744BF42F0200222601BB9226822F045
:104B5000200222601022B1E77546B3FBF2F002FB9F
:104B60001033CB5C05F8013D03460028F5D1B7E7CB
:104B700008681A68496910F0800F04D0101D186089
:104B80001368196007E010F0400F02F1040018608C
:104B90001368F6D01980002323617546B1E71A68BF
:104BA000111D1960156862680021284600F080F820
:104BB00008B1401B606063682361002384F84330C0
:104BC0009FE723692A4639463046C0470130A2D0C4
:104BD00023689B0707D5002504F11909E368039AA8
:104BE0009B1A9D4205DBE068039B9842B8BF1846BC
:104BF00093E701234A4639463046C04701308AD000
:104C00000135EBE7002BA7D10B7884F8423004F193
:104C1000420565E75E5300084D53000810B50C4689
:104C2000B1F90E10FBF7D2FA0028ABBF636DA38970
:104C30001B1823F48053ACBF6365A38110BD2DE91D
:104C4000F0411F468B89DB0505460C46164605D507
:104C500002230022B1F90E10FBF7C5FAA389B4F9BB
:104C60000E1023F48053A38132463B462846BDE80C
:104C7000F041FBF7AFBA10B50C46B1F90E10FBF7D7
:104C8000B2FA431CA38915BF606523F4805343F433
:104C90008053A38118BFA38110BDB1F90E10FBF79B
:104CA0009DBA0000000000000000000000000000AD
:104CB00001F0FF01102A2BDB10F0070F08D010F8CD
:104CC000013B013A8B422DD010F0070F42B3F6D1D1
:104CD000F0B441EA012141EA014122F007047FF0EA
:104CE00000070023F0E80256083C85EA010586EA41
:104CF000010685FA47F5A3FA87F586FA47F6A5FA7D
:104D000087F68EB9EED1F0BC01F0FF0102F0070288
:104D100032B110F8013B013A83EA010313B1F8D133
:104D20000020704701387047002D06BF3546033814
:104D3000073815F0010F07D1013015F4807F02BF4D
:104D4000013015F4C03F0130F0BC0138704700BF9E
:104D500070477047425553204641554C54204841B6
:104D60004E444C4552004445425547204D4F4E203D
:104D700048414E444C45520044554D4D5920484100
:104D80004E444C4552000A49535220737461636B80
:104D9000206F766572666C6F77656400537461632B
:104DA0006B20706F696E74657220636F72727570BC
:104DB0007465642C20726573657420746F20746F41
:104DC00070206F6620737461636B000A436F6E74AA
:104DD000657874206265666F7265206861726466CA
:104DE00061756C743A0020202072303A20307825AA
:104DF00030386C780A20202072313A203078253003
:104E0000386C780A20202072323A203078253038E9
:104E10006C780A20202072333A2030782530386CA4
:104E2000780A0020207231323A2030782530386CF0
:104E3000780A2020206C723A2030782530386C783F
:104E40000A20202070633A2030782530386C780AA8
:104E500020207073723A2030782530386C780A0A36
:104E6000004653522F4641523A0020434653523A8D
:104E70002030782530386C780A0020484653523A62
:104E80002030782530386C780A0020444653523A56
:104E90002030782530386C780A0020414653523A49
:104EA0002030782530386C780A0020424641523A4A
:104EB0002030782530386C780A004D4D4641523A02
:104EC0002030782530386C780A004D6973630045CE
:104ED00058435F5245543A2030782530386C780A70
:104EE00000417474656D7074696E6720746F207210
:104EF00065636F6E73747275637420737461746527
:104F000020666F7220646562756767696E672E2E12
:104F10002E00496E204744423A0A202073657420CF
:104F20002470633D3078256C780A20206672616DAC
:104F30006520300A202062740A000A495352207307
:104F40007461636B206F766572666C6F7765642041
:104F50006279206174206C6561737420256420621D
:104F6000797465732E0A0048415244204641554CDD
:104F7000542048414E444C4552004D454D204D4132
:104F80004E4147452048414E444C4552004E4D4904
:104F90002048414E444C4552005553414745204618
:104FA00041554C542048414E444C455200464149DD
:104FB0004C454420415353455254494F4E2E0025F1
:104FC000700A002A2A2A2052494F54206B65726EBB
:104FD000656C2070616E69633A0A25730A0A002ABB
:104FE0002A2A2068616C7465642E0A0A006D616962
:104FF0006E28293A20546869732069732052494FFA
:105000005421202856657273696F6E3A2032303110
:10501000372E30312D646576656C2D3235352D6730
:1050200031666232312D56616E64726973290A00ED
:1050300069646C65006D61696E00496E73696465D1
:10504000206973722025640A0000000000440040BB
:105050000000020003000240020002400700260692
:10506000040000000048004000000400090C024059
:10507000080C024007002703040000005F5173740E
:10508000617465006E616D650009706964207C2043
:10509000252D3231737C20252D397351207C2070D1
:1050A0007269207C20737461636B2028207573659E
:1050B0006429207C2062617365202020202020202C
:1050C0007C2063757272656E74202020200A0009AE
:1050D00020202D207C206973725F737461636B20C4
:1050E00020202020202020202020207C202D202057
:1050F0002020202020202D207C2020202D207C20DE
:10510000253569202825356929207C2025313070F6
:10511000207C20253130700A000925336869207C05
:1051200020252D323073207C20252D387320252E0C
:105130003173207C20253369207C20253569202887
:1051400025356929207C2025313070207C202531AF
:105150003070200A007C0053554D0009253573201E
:10516000252D3231737C2531337325367320253557
:10517000692028253569290A0073746F7070656489
:1051800000736C656570696E6700626C206D757484
:10519000657800626C20727800626C2073656E64C2
:1051A00000626C207265706C7900626C20616E79AF
:1051B000666C00626C20616C6C666C0072756E6E61
:1051C000696E670070656E64696E6700000000407C
:1051D000FFFFFFFF01000000001C0000000C00406A
:1051E000FFFFFFFF08000000003200000003000086
:1051F000060C024002100240070C02400A0C02405A
:10520000496E697469616C697A696E6720415438C6
:1052100036524632787820726164696F206174205A
:105220005350495F25690A006174383672663278D6
:105230007800415438365246327878206465766971
:105240006365206472697665722074657374000109
:105250000203040202020202020400004F1F0008BF
:10526000D51E0008711E0008BD1D0008BD1F0008E6
:105270005D1B00080F0F0F0E0E0E0E0D0D0C0C0B0C
:105280000B0A0908070605030000030003000200DB
:105290000200010001000000FFFFFEFFFDFFFCFF18
:1052A000FBFFF9FFF7FFF4FFEFFF676E72635F6EBE
:1052B0006574646576323A20706F737369626C79D5
:1052C000206C6F737420696E746572727570742EC1
:1052D00000FFFF0100000000540200200000000059
:1052E00000000000000000000000000000000000BE
:1052F00000000000000000000000000000000000AE
:10530000000000000000000000000000000000009D
:10531000000000000000000000000000000000008D
:10532000000000000000000000000000000000007D
:10533000000000000000000000000000232D302BC2
:105340002000686C4C006566674546470030313286
:1053500033343536373839414243444546003031DD
:10536000323334353637383961626364656600003C
:1053700010280020000000008C03002040000000E6
:105380000000000000000000305000083550000808
:10539000FF00000079510008815100088A5100087F
:1053A0009351000899510008A1510008AA51000822
:1053B000B351000800000000BC510008C4510008AF
:1053C0005402002000000000FC5200081C5300089A
:1053D000DC52000800000000000000000000000097
:1053E00000000000000000000000000000000000BD
:1053F00000000000000000000000000000000000AD
:10540000000000000000000000000000000000009C
:10541000000000000000000000000000000000008C
:045420000000000088
:04000005080004816A
:00000001FF
